:0200000089284D
:0E0006008312031321088A00200882000800DC
:1000140083120313F8010830FC00700DF80D740806
:10002400F80203181728F8070310F00DFC0B0F282B
:020034000800C2
:10003600831603139818212800001B288312310801
:040046009900080015
:10004A0083120313AF0103302F02031833282F083A
:10005A002E07840020308000AF0A28282F082E0798
:10006A0084008001AF032F082E07B0000A30F40085
:10007A002D08F0000A207808F0003030F007300828
:10008A008400700880000A30F4002D08F0000A206D
:10009A007008AD007008003A031D54285628AF03B3
:0400AA0038280800EA
:1000AE0083120313AF012D0884000008AE002E0842
:1000BE00003A03196C282E08B1001B20AF0A2F0836
:0C00CE002D0784000008AE005E2808002A
:1000DA0003208A110A128000840AA00A0319A10ABD
:0800EA00F003031D6D2808005E
:1000F200831603139816903083129800831687177D
:10010200071383128C1E88281A08F0008228080020
:10011200223083120313A6001830A7004230A80031
:100122004630A9003730AA005330AB003030AC0063
:10013200333083169900181579200230FB00043001
:10014200FC00BA30FD00FD0BA428FC0BA428FB0B1D
:10015200A42800002A30A5002508840002300007E8
:10016200AD002230AE0025202230AD0057200B30EA
:10017200FB002630FC005D30FD00FD0BBE28FC0BB1
:0E018200BE28FB0BBE2800000000B528C728D1
:04400E00F22F000786
:00000001FF
